:1000000000308A0004280000FF238316900000308F
:100010008A006928A101A201A001A3012F08031DE4
:1000200014282E0803192E281030B0000310AC0D30
:10003000AD0DA00DA30D2F082302031D21282E08AE
:100040002002031C2A282E08A002031CA3032F0849
:10005000A3020314A10DA20DB00B16280034A001B9
:10006000A1012C0803102D18A007A00CA10CAD189D
:10007000A007A00CA10C2D19A007A00CA10CAD1974
:10008000A007A00CA10C2D1AA007A00CA10CAD1A62
:10009000A007A00CA10C2D1BA007A00CA10CAD1B50
:1000A000A007A00CA10CCE282D30840083130008DB
:1000B000031968280130A100A001A00B5D28A10B45
:1000C0005C284A30A000A00B63286628800B5A28C1
:1000D0000034840183131F3083051F1383161F1000
:1000E0009F101F119F110730831299002710A7102E
:1000F0001F1383161F149F101F119F111F169F1689
:100100001F1383129F171F1483160108C73908385D
:10011000810083129001073099008316050803308F
:100120008312A000A00B922819088C118316990144
:100130008510831285140030A1001F08F3392104B3
:100140009F000330A000A00BA3289F149F18A6288F
:1001500083161E088312A5001E08A60083168510AC
:10016000831285104030AD00C730AC002608AF00C8
:100170002508AE000A202208A6002108A5002608AE
:10018000AD002508AC00AF010A30AE000A202108FE
:10019000AA002A08AC000A30AD002F282108250249
:1001A000AB00271842292714A9010130A800A9088B
:1001B000031D042928082A02031C0429831605119B
:1001C00083120515831685128312851683168510F2
:1001D000831285146430AD005420831605118312F8
:1001E00005118316851283128512831685108312DA
:1001F00085100230AC00C830AD005420AC0BFB2899
:10020000A80A0319A90AD7280430AC00FA30AD00B7
:100210005420AC0B0629A9010130A800A908031D30
:100220003B2928082B02031C3B2983160511831246
:100230000515831685128312851683168510831281
:1002400085146430AD005420831605118312051106
:1002500083168512831285128316851083128510EA
:100260000230AC00C830AD005420AC0B3229A80AD3
:100270000319A90A0E290430AC00FA30AD0054204D
:10028000AC0B3D29A7189229A608031D582925085B
:10029000273C031C58298316051183120515831664
:1002A0008512831285168316851083128514922970
:1002B0002508283C031D8629A608031D86298316C8
:1002C0000511831205158316851283128516831670
:1002D0008510831285140230AC00C830AD00542064
:1002E000AC0B6D2983160511831205118316851237
:1002F0008312851283168510831285100430AC009A
:10030000FA30AD005420AC0B8029922983160511D8
:1003100083120511831685128312851283168510A8
:1003200083128510A714A9010130A800A908031D94
:10033000AB292808643C031CAB298316851583125E
:100340008519A7104230A000A00BA4290000A80A1C
:100350000319A90A9629A71C272AA9010130A80078
:10036000A908031DD9292808053C031CD92983168F
:1003700005118312051583168512831285168316BF
:100380008510831285146430AD0054208316051146
:100390008312051183168512831285128316851028
:1003A000831285103230AD005420A80A0319A90A1F
:1003B000B029A9010130A800A908031D052A2808B1
:1003C000053C031C052A83160511831205158316A7
:1003D0008512831285168316851083128514C83002
:1003E000AD00542083160511831205118316851262
:1003F0008312851283168510831285106430AD0038
:100400005420A80A0319A90ADC29831605118312AE
:10041000051583168512831285168316851083129F
:1004200085140830AC00FA30AD005420AC0B132A10
:100430008316051183120511831685128312851206
:100440008316851083128510C830AD0054208316A2
:1004500098286300FF3FFF3FFF3FFF3FFF3FFF3F05
:10046000FF3FFF3FFF3FFF3FFF3FFF3FFF3FFF3F9C
:10047000FF3FFF3FFF3FFF3FFF3FFF3FFF3FFF3F8C
:10048000FF3FFF3FFF3FFF3FFF3FFF3FFF3FFF3F7C
:10049000FF3FFF3FFF3FFF3FFF3FFF3FFF3FFF3F6C
:1007F000FF3FFF3FFF3FFF3FFF3FFF3FFF3F3C34D7
:02400E00C431BB
:00000001FF
